:100000000C948B000C94A8000C94A8000C94A800ED
:100010000C94A8000C94A8000C94A8000C94A800C0
:100020000C94A8000C94C3080C941B080C94A6080C
:100030000C946C080C9489080C94FE070C944F08DF
:100040000C94B7070C94A8000C94B4090C94A80065
:100050000C949A0A0C94EE020C94A8000C94A8003C
:100060000C94A8000C94A8000C94A8000C94A80070
:100070000C94A8000C94A8000C94A5090C94A8005A
:100080000C948B0A0C94A8000C94A800084AD73B47
:100090003BCE016E84BCBFFDC12F3D6C74319ABD57
:1000A00056833DDA3D00C77F11BED9E4BB4C3E917B
:1000B0006BAAAABE000000803F66693A25642E251F
:1000C000642E256420202B2D2025642E25642E25CA
:1000D00064200D0A00696E6B6C696E6F6D657472D9
:1000E00020323030390D0A00303132333435363772
:1000F00038394142434445460000000100080040B1
:100100000000010004000001000800200040008001
:1001100000000100040011241FBECFEFD0E1DEBFBC
:10012000CDBF12E0A0E0B1E0E8EBFBE202C0059039
:100130000D92A830B107D9F713E0A8E0B2E001C0F2
:100140001D92A337B107E1F70E947E010C94DA15E6
:100150000C9400006F927F928F929F92AF92BF9209
:10016000CF92DF92EF92FF920F931F93CF93DF9383
:100170003B014C0169012115310509F456C05A01B2
:10018000C0E0D0E00F2EF0E0EF2EF0E0FF2EF0E028
:100190000F2FF0E01F2FF02DA4019301F5016191C5
:1001A0007191819191915F010E94210D0E9427150B
:1001B0009B01AC01C801B7010E94520D7B018C016B
:1001C0002196CC15DD0540F30894C108D108B6018D
:1001D00080E090E00894C11CD11C0E9405109B0196
:1001E000AC01C801B7010E94790E0E94DD147B01A9
:1001F0008C01B60180E090E00E9405100E94DD14A1
:100200009B01AC01C801B7010E94790EDF91CF912B
:100210001F910F91FF90EF90DF90CF90BF90AF9024
:100220009F908F907F906F9008950F2EF0E0EF2EAB
:10023000F0E0FF2EF0E00F2FF0E01F2FF02DC4CFE5
:100240008F929F92AF92BF92CF92DF92EF92FF92E6
:100250000F931F936A015901480120E030E044E305
:1002600053E40E947F0D2BED3FE049E450E40E94EF
:10027000790E7B018C010E942A150E94AC0BF601BD
:100280007183608380E090E00E9405109B01AC01C7
:10029000C801B7010E94210D20E030E040E752E4A0
:1002A0000E947F0D7B018C010E942A150E94AC0BDD
:1002B000F501608370E0882777FD8095982F0E9474
:1002C000530F9B01AC01C801B7010E94210D20E032
:1002D00030E040E752E40E947F0D0E94B9140E9472
:1002E000AC0BF40160831F910F91FF90EF90DF90B2
:1002F000CF90BF90AF909F908F9008952F923F9294
:100300004F925F926F927F928F929F92AF92BF9225
:10031000CF92DF92EF92FF920F931F93DF93CF93D1
:10032000CDB7DEB7C850D1400FB6F894DEBF0FBED0
:10033000CDBF0E94A70B40E855E260E070E080E08E
:100340000E94EC0881E599E00E94AE030E94E3055B
:100350000E94A602109261001092620087E00E9443
:10036000B90280E00E94BE0285ED90E09F938F93DA
:1003700081E08F930E942305882499240F900F9089
:100380000F9049E0242E312C2C0E3D1E39E0432ED7
:1003900031E0532E4C0E5D1E30E48316910408F4B8
:1003A0009DC0810160E070E080E090E0F801219163
:1003B0003191419151918F010E94520D0415150503
:1003C000A9F720E030E040E85CE30E947F0D2BEDD0
:1003D0003FE049E450E40E94520D3B014C015101C1
:1003E0000F2EF0E0CF2EF0E0DF2EF0E0EF2EF0E069
:1003F000FF2EF02DA4019301F5016191719181917E
:1004000091915F010E94210D0E9427159B01AC0173
:10041000C701B6010E94520D6B017C01A016B10606
:1004200049F720E030E04CE752E40E94790E0E9448
:10043000DD146B017C018E010E5F1F4F9E012F5F4B
:100440003F4FAE014B5F5F4FC401B3010E942001DB
:1004500020E030E040E05EE3C701B6010E947F0D7E
:100460008E010C5F1F4F9E012D5F3F4FAE01495F14
:100470005F4F0E9420018C8190E09F938F938B812E
:1004800090E09F938F938F8198859F938F938A811C
:1004900090E09F938F93898190E09F938F938D81BC
:1004A0009E819F938F9329EB30E03F932F9381E0C0
:1004B0008F930E94230584E190E00E949306882494
:1004C00099248DB79EB70F960FB6F8949EBF0FBEB6
:1004D0008DBF30E48316910408F063CF80E00E9462
:1004E000D3027C0181E00E94D302A0E0B0E0BC0115
:1004F000CD010E94051020E030E84FEF53E40E9448
:10050000210D5B016C0100E010E0C801B7010E9401
:10051000051020E030E84FEF53E40E94210DA601C2
:1005200095010E942213F401EE0FFF1FEE0FFF1F33
:1005300021E030E02C0F3D1FE20FF31F6087718731
:10054000828793870894811C911C26CF379A35980F
:1005500086B1887F866086B987B18F73806487B9DA
:100560003D98339A10923E037894089533983798C3
:10057000089596B1987F982B96B9089597B1829572
:10058000880F880F807C9F73982B97B9089597B137
:100590008F71907E892B87B90895349A369A089581
:1005A00086B18074089510923E0397B18F71907E4A
:1005B000892B87B9349A369A3699FECF24B145B142
:1005C000942F80E030E0282B392BC90108950E9438
:1005D000D302969587959695879508951F920F92C9
:1005E0000FB60F9211248F938FEF80933E038F915C
:1005F0000F900FBE0F901F901895FC018FB7F894C5
:10060000718360835383428317821682158214821A
:100610008FBF0895CF93DF93DC016FB7F894EC019F
:100620002C813D812115310509F1FC0186819781DD
:10063000ED91FC911197E80FF91FE0810196ED0112
:100640009F838E834A815B818417950750F42150E4
:100650003040ED013D832C836FBF8E2FDF91CF9112
:100660000895841B950B9F838E83F1CFE0E06FBFCD
:100670008E2FDF91CF910895FC01AFB7F8942481BC
:10068000358162177307A8F486819781860F971FBB
:1006900097838683428153818417950720F0841BBA
:1006A000950B97838683261B370B35832483AFBF37
:1006B000089515821482AFBF0895FC01CB012FB7B6
:1006C000F8942FBF2681378162817381820F931F37
:1006D0000E948B120190F081E02DE80FF91F8081BC
:1006E00008951F93CF93DF93EC01462F1FB7F89423
:1006F0002C813D816A817B8126173707B0F48E817A
:100700009F81820F931F0E948B12E881F981E80F6D
:10071000F91F40838C819D8101969D838C831FBF2F
:100720008FEFDF91CF911F9108951FBF80E0DF9180
:10073000CF911F910895FC018FB7F8948FBF22814C
:10074000338184819581281B390BC9010895FC01EF
:100750008FB7F894158214828FBF08959093090281
:100760008093080208951F93182F8A3041F0E0917A
:100770000802F0910902812F09951F910895E091D7
:100780000802F09109028DE00995E0910802F091CC
:100790000902812F09951F910895CF93DF93EC01F2
:1007A000009721F406C021960E94B3038881882314
:1007B000D1F7DF91CF910895EF92FF920F931F939E
:1007C000CF93DF938C017A01009729F120E030E08C
:1007D0002617370738F4F80181918F012F5F3F4FBB
:1007E0008823B1F7E114F104B1F0C0E0D0E008C013
:1007F0000F5F1F4F0E94B3032196CE15DF0558F4FB
:10080000F80180818823A1F780E20E94B30321963A
:10081000CE15DF05A8F3DF91CF911F910F91FF90C7
:10082000EF900895CF93DF93FC01009761F08491DE
:10083000882349F0EF0121960E94B303FE0121961F
:1008400084918823C9F7DF91CF9108958AE00E94AF
:10085000B3030895E82FF0E0EF70F070E851FF4F18
:10086000E4918E2F0E94B30308951F93182F829551
:100870008F700E942A04812F0E942A041F910895DC
:100880001F93182F892F0E943504812F0E94350451
:100890001F910895EF92FF920F931F937B018C019C
:1008A000C801AA27BB270E944004C7010E94400438
:1008B0001F910F91FF90EF9008952F923F924F92CA
:1008C0005F926F927F928F929F92AF92BF92CF92E0
:1008D000DF92EF92FF920F931F93DF93CF93CDB7E9
:1008E000DEB7A4970FB6F894DEBF0FBECDBF6BA3E3
:1008F000A42E2CA317012801442311F017FD98C042
:10090000820171012BA121502AA390E0A11091E056
:10091000EAA1E91BE9A318A2682E772467FC70946A
:10092000872C972CC801B701A40193010E949F1244
:10093000FB01EF70F070E851FF4F64916F8FC801B9
:10094000B701A40193010E949F12C901DA017C0141
:100950008D019EE1C92ED12CCC0EDD1EB9A01CC08C
:10096000C801B701A40193010E949F12FB01EF701F
:10097000F070E851FF4F6491F6016083C801B70140
:10098000A40193010E949F12C901DA017C018D012B
:10099000BA940894C108D108BB2049F0E114F104CD
:1009A00001051105E9F62CA1F6012083F1CFCE0156
:1009B0004F96FC0129A1E21BF109AA2049F057FC3E
:1009C00034C02114310441045104D1F18BE28293EB
:1009D0008BA1882389F08F019AA1E92EFF24089426
:1009E000E11CF11CEE0EFF1EF80181918F010E94A7
:1009F000B3030E151F05C1F7A4960FB6F894DEBF1A
:100A00000FBECDBFCF91DF911F910F91FF90EF905F
:100A1000DF90CF90BF90AF909F908F907F906F901E
:100A20005F904F903F902F9008958DE28293D0CFAA
:100A3000EE24FF248701E218F3080409150962CFA8
:100A400080E28293C5CF7F928F929F92AF92BF92A6
:100A5000CF92DF92EF92FF920F931F93DF93CF938A
:100A6000CDB7DEB77888C988DA888E010D5E1F4F52
:100A7000772081F0F6010894C11CD11C8491853245
:100A800071F0882309F474C00E94B3034801840103
:100A9000772081F7F60181916F01853291F77720F8
:100AA00081F0F6010894C11CD11C8491843671F048
:100AB0008837D9F1833689F148010E94B303840154
:100AC000E7CFF60181916F01843691F722E0822E03
:100AD000912C800E911EF801E080F180FF200CF433
:100AE00057C0F0E1EF16F7E2FF0608F059C088EEB4
:100AF000E81683E0F80608F059C0E4E6EE16F104C3
:100B000008F05AC0FAE0EF16F10408F058C001E00E
:100B100010E04AE0A42EB12C15C0E2E08E2E912CFC
:100B2000800E911EF8018081C8CF72E0872E912C33
:100B3000800E911EF801E080F18000E010E160E19C
:100B4000A62EB12CC701B8010E948B12862F0E94DD
:100B50002A04C701B8010E948B127C01C801B501AB
:100B60000E948B128B016115710561F7840190CF92
:100B700080E090E0CF91DF911F910F91FF90EF9077
:100B8000DF90CF90BF90AF909F908F907F9008950F
:100B9000F094E194F108F3948DE20E94B303A1CFA5
:100BA00000E117E25AE0A52EB12CCCCF08EE13E0FD
:100BB0003AE0A32EB12CC6CF04E610E0F9CF0AE04C
:100BC00010E0F6CF089580E090E0FC01EE0FFF1FEB
:100BD000E65FFD4F11821082019688309105A9F7DA
:100BE00083B7887F826083BF12BE87B7816087BF6B
:100BF00010923F031092400310924103109242035F
:100C00008EB5887F83608EBD1DBC1CBC87B7846099
:100C100087BF85B5887F846085BD14BC87B7806435
:100C200087BF109247031092480310924903109215
:100C30004A037894089583B7887F826083BF12BE89
:100C400087B7816087BF10923F03109240031092D4
:100C500041031092420308958EB5887F83608EBD54
:100C60001DBC1CBC87B7846087BF089585B5887F8D
:100C7000846085BD14BC87B7806487BF109247032A
:100C8000109248031092490310924A03089593B7B3
:100C9000987F982B93BF08959EB5987F982B9EBD03
:100CA000089595B5987F982B95BD089583B7E82F43
:100CB000F0E0E770F070EE0FFF1FE750FF4F259157
:100CC0003491C90108958EB5E82FF0E0E770F07017
:100CD000EE0FFF1FE750FF4F25913491C901089592
:100CE00085B5E82FF0E0E770F070EE0FFF1FEB5FC7
:100CF000FE4F25913491C9010895883040F4E82FC2
:100D0000F0E0EE0FFF1FE65FFD4F718360830895F3
:100D1000883040F4E82FF0E0EE0FFF1FE65FFD4F54
:100D2000118210820895DF92EF92FF920F931F932A
:100D30008C01D2B6109243031092440310924503E3
:100D40001092460383B7E82FF0E0E770F070EE0FE3
:100D5000FF1FE750FF4F2591349140E050E060E0E5
:100D600072E18AE790E00E94C112B901CA01693BB1
:100D70002DE8720726E0820720E0920728F427E298
:100D80000131120708F44EC028EE33E040E050E095
:100D90000E949F12CA01B901980140E050E00E94F0
:100DA0006C127B018C0120914303309144034091EC
:100DB00045035091460382B7ED0CF11C011D111D36
:100DC0001BC08091430390914403A0914503B091CF
:100DD000460385B7837E85BF85B7806285BF8895CA
:100DE00085B78F7D85BF20914303309144034091A7
:100DF00045035091460382B790E0A0E0B0E0542F45
:100E0000432F322F2227822B932BA42BB52B8E1509
:100E10009F05A007B107A8F21F910F91FF90EF90D7
:100E2000DF900895980140E050E00E946C1228EE97
:100E300033E040E050E00E949F12C901DA017C01DA
:100E40008D01B1CF10923F031092400310924103E5
:100E500010924203089520913F0330914003409146
:100E6000410350914203B901CA010895109247030A
:100E7000109248031092490310924A03089520915A
:100E80004703309148034091490350914A03B90107
:100E9000CA010895893069F08A30B1F08FB58D7F2D
:100EA0008FBD8FB581608FBD1BBC1ABC19BC18BC2F
:100EB00008958FB582608FBD8FB58E7F8FBD1BBCAF
:100EC0001ABC19BC18BC08958FB582608FBD8FB550
:100ED00081608FBD1BBC1ABC19BC18BC08952FB50E
:100EE0002E7F2FBD2FB522602FBD2EB528602EBDC1
:100EF0002EB520612EBD97BD86BD1BBC1ABC19BC8A
:100F000018BC08958FB58D7F8FBD8FB58E7F8FBD37
:100F10008FB58F778FBD8FB58F7B8FBD8FB58F7D51
:100F20008FBD8FB58F7E8FBD08958FB580688FBDC3
:100F30008FB58F7B8FBD08958FB580628FBD8FB5C4
:100F40008F7E8FBD08958FB58F778FBD8FB58F7BC7
:100F50008FBD08958FB58F7D8FBD8FB58F7E8FBD6F
:100F600008959BBD8ABD089599BD88BD08951F92BF
:100F70000F920FB60F9211248F939F93AF93BF934D
:100F8000EF93FF9380913F0390914003A091410321
:100F9000B09142030196A11DB11D80933F03909330
:100FA0004003A0934103B093420380914303909187
:100FB0004403A0914503B09146030196A11DB11DC4
:100FC0008093430390934403A0934503B093460357
:100FD00080910A0290910B02892B29F0E0910A027C
:100FE000F0910B020995FF91EF91BF91AF919F9105
:100FF0008F910F900FBE0F901F9018951F920F9218
:101000000FB60F9211248F939F93EF93FF938091CC
:101010000C0290910D02892B29F0E0910C02F091C5
:101020000D020995FF91EF919F918F910F900FBE47
:101030000F901F9018951F920F920FB60F921124C8
:101040008F939F93AF93BF93EF93FF938091470349
:1010500090914803A0914903B0914A030196A11DC4
:10106000B11D8093470390934803A0934903B09325
:101070004A038091140290911502892B29F0E09186
:101080001402F09115020995FF91EF91BF91AF9174
:101090009F918F910F900FBE0F901F9018951F92E8
:1010A0000F920FB60F9211248F939F93EF93FF939C
:1010B0008091180290911902892B29F0E091180271
:1010C000F09119020995FF91EF919F918F910F90E7
:1010D0000FBE0F901F9018951F920F920FB60F9290
:1010E00011248F939F93EF93FF9380910E02909121
:1010F0000F02892B29F0E0910E02F0910F02099561
:10110000FF91EF919F918F910F900FBE0F901F90C5
:1011100018951F920F920FB60F9211248F939F93E1
:10112000EF93FF938091100290911102892B29F087
:10113000E0911002F09111020995FF91EF919F91BA
:101140008F910F900FBE0F901F9018951F920F92C6
:101150000FB60F9211248F939F93EF93FF9380917B
:10116000120290911302892B29F0E0911202F09162
:1011700013020995FF91EF919F918F910F900FBEF0
:101180000F901F9018951F920F920FB60F92112477
:101190008F939F93EF93FF93809116029091170284
:1011A000892B29F0E0911602F09117020995FF9121
:1011B000EF919F918F910F900FBE0F901F901895F8
:1011C000823008F00895E82FF0E0EE0FFF1FE65C94
:1011D000FC4F7183608308951F93182F9A01AB0110
:1011E000CA01B901605C7D4B804F9F4F660F771F2E
:1011F000881F991F660F771F881F991F660F771F1B
:10120000881F991F220F331F441F551F220F331FA2
:10121000441F551F220F331F441F551F220F331F1A
:10122000441F551F0E949F1221503040112329F462
:1012300029B9309390001F9108952093990030931D
:1012400098001F910895282F30E0220F331F220F9E
:10125000331F220F331F235B3C4FC9010895282FF2
:1012600030E0220F331F220F331F220F331F215A6A
:101270003C4FC9010895E82F882359F080919B00C5
:1012800085FFFCCF60939C00F0E0E55BFC4F108293
:1012900008955D9BFECF6CB9F0E0E55BFC4F1082DA
:1012A00008955D9BFECF8CB910924B030895982F43
:1012B00080919B0085FFFCCF90939C0010924C0383
:1012C000089520E0E82FF0E0EE0FFF1FEE0FFF1F64
:1012D000EE0FFF1FEF5AFC4F80819181892B09F49B
:1012E00021E0822F0895CF93DF938823B1F060919E
:1012F0009C00282F30E0E901CC0FDD1FFE01E65CE9
:10130000FC4F80819181892B51F00190F081E02D7B
:10131000862F0995DF91CF9108956CB1EACF220F06
:10132000331F220F331F220F331FC901835B9C4FD2
:101330000E947103882371F7FE01E159FC4F8081FF
:101340009181019691838083E5CF1F920F920FB612
:101350000F9211248F9381E00E9473098F910F9057
:101360000FBE0F901F9018951F920F920FB60F92FD
:1013700011248F9380E00E9473098F910F900FBE0C
:101380000F901F9018958F929F92AF92BF92CF921D
:10139000DF92EF92FF920F931F93CF93DF93982EDC
:1013A000DB01C82EDD24F601EE0FFF1FEE0FFF1F3D
:1013B000EE0FFF1FED59FC4F20813181240F351FA7
:1013C000F601EE0FFF1FEE0FFF1FEE0FFF1FEF598D
:1013D000FC4F808191812817390790F541155105FF
:1013E00079F18C905A010894A108B108A114B104B4
:1013F000C9F07601EE0CFF1CEE0CFF1CEE0CFF1C7E
:101400008FE593E0E80EF91E8D01C0E0D0E0F80111
:101410006181C7010E94710321960F5F1F4FCA159A
:10142000DB05A8F3F601E35AFC4F8FEF8083992088
:10143000A9F080919B0085FFFCCF80929C0011C099
:1014400080E0DF91CF911F910F91FF90EF90DF909F
:10145000CF90BF90AF909F908F9008955D9BFECFEF
:101460008CB88BE493E0C80ED91EF60110828FEF82
:10147000E8CF90E0880F991F880F991F880F991F58
:10148000815A9C4F0E9471030895682F87E693E06C
:101490000E9471030895682F8FE593E00E94710305
:1014A0000895CF93DF93282FA82FB0E0ED01C35A02
:1014B000DC4F88818823C1F0FD01EE0FFF1FEE0F86
:1014C000FF1FEE0FFF1FED59FC4F80819181892B8B
:1014D00091F02223C1F087E693E00E940A038093F3
:1014E0009C00DF91CF910895A55BBC4F8FEF8C934B
:1014F000DF91CF9108951882A55BBC4F8FEF8C933D
:10150000DF91CF9108958FE593E00E940A038CB993
:10151000DF91CF9108951F920F920FB60F92112471
:101520008F9381E00E94510A8F910F900FBE0F9010
:101530001F9018951F920F920FB60F9211248F9340
:1015400080E00E94510A8F910F900FBE0F901F9064
:1015500018951F93CF93DF93182FC82FD0E0FE016B
:10156000E35AFC4F8FEF8083CE01880F991F880FBD
:10157000991F880F991F815A9C4F0E940A03982F28
:10158000112369F080919B0085FFFCCF90939C0014
:10159000C55BDC4F1882DF91CF911F9108955D9B51
:1015A000FECF9CB9C55BDC4F1882DF91CF911F91B4
:1015B0000895CF93DF93EB01282F30E0F901EE0F70
:1015C000FF1FEE0FFF1FEE0FFF1FE15BFC4F80813F
:1015D0009181892B69F0F901EE0FFF1FEE0FFF1FBC
:1015E000EE0FFF1FEF5AFC4F80819181892B21F470
:1015F00080E0DF91CF910895220F331F220F331F18
:10160000220F331FC901835B9C4F0E940A0388830A
:101610008FEFDF91CF910895DF93CF930F92CDB7E6
:10162000DEB7BE016F5F7F4F81E00E94D90A882339
:1016300041F08981282F30E0C9010F90CF91DF91CF
:1016400008952FEF3FEFC9010F90CF91DF910895DB
:10165000DF93CF930F92CDB7DEB7BE016F5F7F4FA1
:1016600080E00E94D90A882341F08981282F30E048
:10167000C9010F90CF91DF9108952FEF3FEFC9017E
:101680000F90CF91DF91089590E0880F991F880FF8
:10169000991F880F991F835B9C4F0E94A703089591
:1016A00040E850E06AEA72E085E593E00E94FD02BE
:1016B00040E150E06AE273E087E693E00E94FD02B9
:1016C00008950E94500B10923D0310923C0388ED48
:1016D00080939A0040E855E260E070E081E00E946B
:1016E000EC088FEF80934C0310925E03109272030C
:1016F000109271037894089540E850E06AE172E036
:101700008DE493E00E94FD0240E150E06AE972E05E
:101710008FE593E00E94FD0208950E947C0B1092D9
:101720003B0310923A0388ED8AB940E855E260E045
:1017300070E080E00E94EC088FEF80934B031092E2
:101740005D031092700310926F03789408950E94C5
:101750008D0B0E94610B0895EF92FF920F931F93E0
:101760007B018C0120E030E040E05FE40E94230F29
:1017700088238CF020E030E040E05FE4C801B7014E
:101780000E94210D0E94B10F9B01AC0120503040FE
:101790004040504806C0C801B7010E94B10F9B01EC
:1017A000AC01B901CA011F910F91FF90EF9008950C
:1017B000A0E0B0E0EEEDFBE00C94DC12DC012B01CC
:1017C000FA019C91923008F436C1EB018881823095
:1017D00008F430C1943061F4843009F02CC1FD016B
:1017E00091818981981709F426C1A0E0B1E023C155
:1017F000843009F41FC18230A9F4923009F01BC172
:101800009A01AD0188E0EA010990AE01E90109926F
:101810009E018150C1F7E2018981ED0199818923FF
:10182000818306C1923009F405C1ED012A803B8015
:10183000EB018A819B81ED01AC80BD80CE80DF8091
:10184000EB01EC80FD800E811F819101281B390B7B
:10185000B90137FF04C066277727621B730B60321C
:1018600071050CF061C0121613066CF537014801C2
:10187000062E04C096948794779467940A94D2F7BE
:1018800021E030E040E050E004C0220F331F441F4D
:10189000551F6A95D2F721503040404050402E21CC
:1018A0003F2140235123211531054105510521F0E8
:1018B00021E030E040E050E079018A01E628F72895
:1018C000082919293CC0232BD1F1260E371E3501DA
:1018D0004601062E04C096948794779467940A94E0
:1018E000D2F721E030E040E050E004C0220F331F87
:1018F000441F551F6A95D2F7215030404040504058
:101900002A213B214C215D2121153105410551053D
:1019100021F021E030E040E050E059016A01A628C2
:10192000B728C828D9280BC0821593052CF01C01B4
:10193000AA24BB24650103C0EE24FF248701ED0126
:101940009981E2018981981709F445C0992339F0FA
:10195000A80197012A193B094C095D0906C0A60197
:1019600095012E193F09400B510B57FD08C01182FC
:101970003382228224833583468357831DC081E0CE
:1019800081833382228288279927DC01821B930B73
:10199000A40BB50B84839583A683B7830DC0220F58
:1019A000331F441F551F2483358346835783828109
:1019B0009381019793838283248135814681578166
:1019C000DA01C9010197A109B1098F5F9F4FAF4F9C
:1019D000BF4328F30BC0918333822282EA0CFB1CA5
:1019E0000C1D1D1DE482F5820683178383E080832E
:1019F000248135814681578157FF1AC0C901AA2722
:101A000097FDA095BA2F81709070A070B070569518
:101A1000479537952795822B932BA42BB52B848341
:101A20009583A683B7838281938101969383828372
:101A3000DF0101C0D201CD01CDB7DEB7E2E10C94E8
:101A4000F812A0E2B0E0E7E2FDE00C94E81269834E
:101A50007A838B839C832D833E834F835887E9E071
:101A6000EE2EF12CEC0EFD1EB701CE0101960E9468
:101A7000A2118E010F5E1F4FB801CE0105960E9484
:101A8000A2118A8991E089278A8BAE01475E5F4F58
:101A9000B801C7010E94D80B0E94CD10A096E6E0C5
:101AA0000C940413A0E2B0E0E8E5FDE00C94E81229
:101AB00069837A838B839C832D833E834F835887EE
:101AC000F9E0EF2EF12CEC0EFD1EB701CE010196D0
:101AD0000E94A2118E010F5E1F4FB801CE01059624
:101AE0000E94A211AE01475E5F4FB801C7010E947C
:101AF000D80B0E94CD10A096E6E00C940413A0E24F
:101B0000B0E0E5E8FDE00C94DC1269837A838B8316
:101B10009C832D833E834F835887BE01675F7F4F31
:101B2000CE0101960E94A211BE016F5E7F4FCE01D1
:101B300005960E94A2119985923088F08989823099
:101B4000C8F0943019F4823051F404C0843029F480
:101B5000923081F480E091E0C6C0923049F420E0F8
:101B60009A858A89981321E02A87CE010996BBC0FD
:101B7000823049F420E09A858A89981321E02A8BE3
:101B8000CE014196B0C02D843E844F8458886D8824
:101B90007E888F88988CEE24FF248701AA24BB249A
:101BA000650140E050E060E070E0E0E0F0E0C1019D
:101BB00081709070892BE9F0E60CF71C081D191D47
:101BC0009A01AB012A0D3B1D4C1D5D1D80E090E08C
:101BD000A0E0B0E0E614F7040805190520F481E060
:101BE00090E0A0E0B0E0BA01A901480F591F6A1FB8
:101BF0007B1FAA0CBB1CCC1CDD1C97FE08C081E01F
:101C000090E0A0E0B0E0A82AB92ACA2ADB2A3196DF
:101C1000E032F10549F0660C771C881C991C56943B
:101C2000479437942794C3CFFA85EA892B893C8956
:101C30008B859C85280F391F2E5F3F4F17C0CA0127
:101C400081709070892B61F016950795F794E79451
:101C500080E090E0A0E0B0E8E82AF92A0A2B1B2BEC
:101C600076956795579547952F5F3F4F77FDE7CF5F
:101C70000CC0440F551F661F771F17FD4160EE0C07
:101C8000FF1C001F111F21503040403090E05907C9
:101C900090E0690790E4790760F32B8F3C8FDB01BC
:101CA000CA018F779070A070B07080349105A10543
:101CB000B10561F447FD0AC0E114F1040105110505
:101CC00029F0405C5F4F6F4F7F4F40781A8EFE17B0
:101CD00011F081E08A8F4D8F5E8F6F8F78A383E044
:101CE000898FCE0149960E94CD10A096E2E10C9416
:101CF000F812A8E1B0E0EFE7FEE00C94E41269838B
:101D00007A838B839C832D833E834F835887B9E0EE
:101D1000EB2EF12CEC0EFD1EB701CE0101960E94B8
:101D2000A2118E010F5E1F4FB801CE0105960E94D1
:101D3000A2112985223008F47CC03989323010F490
:101D4000B8017AC08A859A8989278A87243011F058
:101D5000223031F4231709F06CC060E071E06CC0F0
:101D6000343039F41D861E861F86188A1C861B8611
:101D700004C0323021F484E08987B7015DC02B852F
:101D80003C858B899C89281B390B3C872B87ED84EC
:101D9000FE840F851889AD88BE88CF88D88CEA1458
:101DA000FB040C051D0540F4EE0CFF1C001F111F69
:101DB000215030403C872B8720E030E040E050E06D
:101DC00080E090E0A0E0B0E46FE170E0EA14FB0492
:101DD0000C051D0540F0282B392B4A2B5B2BEA18EC
:101DE000FB080C091D09B695A79597958795EE0CEC
:101DF000FF1C001F111F6150704041F7DA01C9013B
:101E00008F779070A070B07080349105A105B105F6
:101E100061F427FD0AC0E114F1040105110529F060
:101E2000205C3F4F4F4F5F4F20782D873E874F8775
:101E3000588BBE01675F7F4FCB010E94CD10689623
:101E4000EAE00C940013A8E1B0E0E9E2FFE00C94B2
:101E5000E81269837A838B839C832D833E834F832F
:101E6000588789E0E82EF12CEC0EFD1EB701CE015B
:101E700001960E94A2118E010F5E1F4FB801CE0184
:101E800005960E94A2118985823040F089898230AE
:101E900028F0B801C7010E94121201C08FEF6896A6
:101EA000E6E00C940413A8E0B0E0E9E5FFE00C9450
:101EB000E5129B01AC0183E08983DA01C90188271F
:101EC000B7FD83959927AA27BB27B82E2115310581
:101ED0004105510519F482E089833AC08823A9F0AD
:101EE000203080E0380780E0480780E8580729F470
:101EF00060E070E080E09FEC30C0EE24FF248701BA
:101F0000E21AF30A040B150B02C079018A018EE173
:101F1000C82ED12CDC82CB82ED82FE820F83188703
:101F2000C801B7010E947E1001971816190684F4A3
:101F3000082E04C0EE0CFF1C001F111F0A94D2F7DC
:101F4000ED82FE820F831887C81AD90ADC82CB8201
:101F5000BA82CE0101960E94CD102896E9E00C9439
:101F60000113ACE0B0E0E7EBFFE00C94EC12698306
:101F70007A838B839C83BE016B5F7F4FCE0101967A
:101F80000E94A2118D81823061F1823050F1843043
:101F900021F48E81882351F12EC02F81388537FDA1
:101FA00020C06E812F3131051CF06623F9F023C06B
:101FB0008EE190E0821B930B29853A854B855C85E9
:101FC00004C056954795379527958A95D2F766238D
:101FD000B1F050954095309521953F4F4F4F5F4F51
:101FE0000EC020E030E040E050E009C02FEF3FEFAE
:101FF0004FEF5FE704C020E030E040E050E8B90177
:10200000CA012C96E2E00C940813A8E0B0E0EBE0E3
:10201000F0E10C94E6127B018C01611571058105DC
:10202000910519F482E0898360C083E089838EE1A1
:10203000C82ED12CDC82CB82ED82FE820F831887E2
:10204000C801B7010E947E10BC016150704077FF4B
:1020500039C0EE27FF27E61BF70B20E030E040E019
:1020600050E081E090E0A0E0B0E00E2E04C0880FC8
:10207000991FAA1FBB1F0A94D2F70197A109B109A2
:102080008E219F21A023B1230097A105B10521F046
:1020900021E030E040E050E004C016950795F79449
:1020A000E794EA95D2F72E293F29402B512B2D8317
:1020B0003E834F8358878EE190E0861B970B9C836D
:1020C0008B8313C06115710581F0062E04C0EE0CE0
:1020D000FF1C001F111F0A94D2F7ED82FE820F83AE
:1020E0001887C61AD70ADC82CB821A82CE010196E3
:1020F0000E94CD102896E8E00C940213EF92FF9214
:102100000F931F937B018C0180E0E81680E0F806B6
:1021100081E0080780E0180788F48FEFE816F104E3
:102120000105110531F028F088E090E0A0E0B0E072
:1021300017C080E090E0A0E0B0E012C080E0E816B8
:1021400080E0F80680E0080781E0180728F088E1C1
:1021500090E0A0E0B0E004C080E190E0A0E0B0E05A
:1021600020E230E040E050E0281B390B4A0B5B0BCB
:1021700004C016950795F794E7948A95D2F7F7016E
:10218000E85FFE4F8081281B310941095109C901CF
:102190001F910F91FF90EF900895DF92EF92FF92C1
:1021A0000F931F93FC01E480F58006811781D18095
:1021B0008081823048F480E090E0A0E1B0E0E82A3D
:1021C000F92A0A2B1B2BA5C0843009F49FC082304A
:1021D00021F4EE24FF24870105C0E114F104010578
:1021E000110519F4E0E0F0E096C0628173819FEF81
:1021F000623879070CF05BC022E83FEF261B370BF3
:102200002A3131052CF020E030E040E050E02AC0D7
:10221000B801A701022E04C076956795579547959A
:102220000A94D2F781E090E0A0E0B0E004C0880F0B
:10223000991FAA1FBB1F2A95D2F70197A109B109BF
:102240008E219F21A023B1230097A105B10521F084
:1022500081E090E0A0E0B0E09A01AB01282B392B9F
:102260004A2B5B2BDA01C9018F779070A070B07098
:1022700080349105A105B10539F427FF09C0205C20
:102280003F4F4F4F5F4F04C0215C3F4F4F4F5F4F59
:10229000E0E0F0E02030A0E03A07A0E04A07A0E448
:1022A0005A0710F0E1E0F0E079018A0127C06038B8
:1022B000710564F5FB01E158FF4FD801C7018F7725
:1022C0009070A070B07080349105A105B10539F40B
:1022D000E7FE0DC080E490E0A0E0B0E004C08FE332
:1022E00090E0A0E0B0E0E80EF91E0A1F1B1F17FFE8
:1022F00005C016950795F794E794319687E01695F3
:102300000795F794E7948A95D1F705C0EE24FF244A
:102310008701EFEFF0E06E2F679566276795902FA6
:102320009F77D794DD24D7948E2F8695492F462BFF
:10233000582F5D29B701CA011F910F91FF90EF90AF
:10234000DF900895FC01DB01408151812281622FE1
:102350006F7770E0221F2227221F9381892F880F19
:10236000822B282F30E0991F9927991FFD01918317
:102370002115310581F5411551056105710511F4EE
:1023800082E032C082E89FEFFD01938382839A014D
:10239000AB0167E0220F331F441F551F6A95D1F729
:1023A00083E08C930AC0220F331F441F551FFD0189
:1023B000828193810197938382832030F0E03F07ED
:1023C000F0E04F07F0E45F0770F3FD0124833583ED
:1023D0004683578308952F3F310581F441155105F8
:1023E0006105710519F484E08C93089564FF03C0BE
:1023F00081E08C9301C01C92FD010FC02F5730402B
:10240000FD013383228383E08C9387E0440F551FC3
:10241000661F771F8A95D1F770644483558366835E
:10242000778308951F93CF93DF93DC01FB019C9189
:10243000923008F444C08081823008F440C0943067
:1024400051F4ED011981843081F58181682F70E0AC
:10245000611B71093CC0843021F0923031F482302C
:10246000A1F18181882371F12AC0ED0119818230A7
:10247000E1F081811817C9F4ED012A813B81828145
:102480009381821793078CF028173907B4F0ED0178
:102490008C819D81AE81BF812481358146815781A8
:1024A000281739074A075B0718F4112341F00AC0BF
:1024B00082179307A407B50740F4112319F061E0D0
:1024C00070E005C06FEF7FEF02C060E070E0CB010D
:1024D000DF91CF911F910895629FD001739FF0010A
:1024E000829FE00DF11D649FE00DF11D929FF00DA4
:1024F000839FF00D749FF00D659FF00D9927729FDB
:10250000B00DE11DF91F639FB00DE11DF91FBD0165
:10251000CF0111240895AA1BBB1B51E107C0AA1FBC
:10252000BB1FA617B70710F0A61BB70B881F991F74
:102530005A95A9F780959095BC01CD010895A1E227
:102540001A2EAA1BBB1BFD010DC0AA1FBB1FEE1F2D
:10255000FF1FA217B307E407F50720F0A21BB30B78
:10256000E40BF50B661F771F881F991F1A9469F7F4
:1025700060957095809590959B01AC01BD01CF0150
:10258000089597FB092E05260ED057FD04D0D7DFFE
:102590000AD0001C38F450954095309521953F4F56
:1025A0004F4F5F4F0895F6F7909580957095619520
:1025B0007F4F8F4F9F4F08952F923F924F925F9280
:1025C0006F927F928F929F92AF92BF92CF92DF9243
:1025D000EF92FF920F931F93CF93DF93CDB7DEB7A8
:1025E000CA1BDB0B0FB6F894DEBF0FBECDBF09943C
:1025F0002A88398848885F846E847D848C849B8493
:10260000AA84B984C884DF80EE80FD800C811B81A0
:10261000AA81B981CE0FD11D0FB6F894DEBF0FBECF
:10262000CDBFED010895F5D058F080E891E009F4B0
:102630009EEFF6D028F040E851E059F45EEF09C073
:10264000C0C028C1E92FE07803D168F3092E052A1C
:10265000C1F3261737074807590738F00E2E07F839
:10266000E02569F0E025E0640AC0EF6307F8009414
:1026700007FADB01B9019D01DC01CA01AD01EF934D
:1026800041D0D5D00AD05F91552331F02BED3FE0FA
:1026900049E450FD49EC06CA0895DF93DD27B92FC0
:1026A000BF7740E85FE31616170648075B0710F48C
:1026B000D92FF7D09F938F937F936F93C8D1ECE876
:1026C000F0E082D0B4D02F913F914F915F91FAD03A
:1026D000DD2349F09058A2EA2AED3FE049EC5FE3A0
:1026E000D0785D27CBD1DF91A2C09AD040F091D0B5
:1026F00030F021F45F3F19F05EC05111CCC061C0D1
:10270000A7D098F39923C9F35523B1F3951B550B23
:10271000BB27AA2762177307840738F09F5F5F4FB4
:10272000220F331F441FAA1FA9F333D00E2E3AF0F5
:10273000E0E830D091505040E695001CCAF729D00F
:10274000FE2F27D0660F771F881FBB1F261737075E
:102750004807AB07B0E809F0BB0B802DBF01FF278E
:1027600093585F4F2AF09E3F510568F024C093C0F4
:102770005F3FECF3983EDCF3869577956795B795C8
:10278000F7959F5FC9F7880F911D9695879597F9E3
:102790000895E1E0660F771F881FBB1F621773075C
:1027A0008407BA0720F0621B730B840BBA0BEE1F71
:1027B00088F7E095089597F99F6780E870E060E0FA
:1027C00008959FEF80EC0895DF93CF931F930F93AD
:1027D000FF92EF92DF927B018C01689405C0DA2EA4
:1027E000EF0170D0FE01E894A591259135914591B6
:1027F0005591AEF3EF0142D1FE019701A801DA94A1
:1028000079F7DF90EF90FF900F911F91CF91DF91BB
:10281000089500240A941616170618060906089546
:1028200000240A9412161306140605060895092EAC
:102830000394000C11F4882352F0BB0F40F4BF2B1B
:1028400011F460FF04C06F5F7F4F8F4F9F4F08955B
:1028500057FD9058440F551F59F05F3F71F0479551
:10286000880F97FB991F61F09F3F79F08795089536
:10287000121613061406551FF2CF4695F1DF08C055
:10288000161617061806991FF1CF86957105610572
:1028900008940895E894BB2766277727CB0197F91A
:1028A00008959B01AC0160E070E080E89FE321CADD
:1028B000B0DF28F0B5DF18F0952309F07CCF81CF89
:1028C0001124E9CFC5DFA0F3959FD1F3950F50E018
:1028D000551F629FF001729FBB27F00DB11D639FD2
:1028E000AA27F00DB11DAA1F649F6627B00DA11D78
:1028F000661F829F2227B00DA11D621F739FB00D1E
:10290000A11D621F839FA00D611D221F749F33278D
:10291000A00D611D231F849F600D211D822F762F26
:102920006A2F11249F5750408AF0E1F088234AF023
:10293000EE0FFF1FBB1F661F771F881F915050406F
:10294000A9F79E3F510570F036CFA5CF5F3FECF35E
:10295000983EDCF3869577956795B795F795E7955B
:102960009F5FC1F7FE2B880F911D9695879597F96C
:10297000089576DFE0F09E37D8F09639B8F49E38A7
:1029800048F4672F782F8827985FF9CF8695779539
:10299000679593959539D0F3B62FB1706B0F711D74
:1029A000811D20F48795779567959395BAC0D4C01B
:1029B00072CF11F40EF405CFCFC052DFD0F39923BC
:1029C000D9F3CEF39F57550B87FFD6D056959795E1
:1029D000B0E020F4660F771F881FBB1F1F930F9373
:1029E00000249001A0018001F001A0E80E0F1F1F3C
:1029F0000A1E511D601B710B8009B50B48F4600F56
:102A0000711F801DB51F0E1B1F0B0A0A510907C03D
:102A10002E0F3F1F4A1F0E0F1F1F0A1E511D660F4C
:102A2000771F881FBB1FA695F795E795F8F6061741
:102A3000170708065B07211D311D411D0F911F91CE
:102A4000B901842F9158880F9695879508959B0119
:102A5000AC0155C898D020F09F3708F41CCF61C056
:102A60007BC0D7DE30F0DCDE20F031F49F3F11F484
:102A70001EF4A7CE0EF4E095E7FB9DCEE92FE8DE2D
:102A800080F3BA17620773078407950718F071F48B
:102A90009EF500CF0EF4E0950B2EBA2FA02D0B0162
:102AA000B90190010C01CA01A0011124FF27591B93
:102AB00099F0593F50F4503E68F11A16F040A22F99
:102AC000232F342F4427585FF3CF4695379527950A
:102AD000A795F0405395C9F77EF41F16BA0B620B09
:102AE000730B840BBAF09150A1F0FF0FBB1F661F50
:102AF000771F881FC2F70EC0BA0F621F731F841F93
:102B000048F4879577956795B795F7959E3F08F0B8
:102B1000B3CF9395880F08F09927EE0F9795879577
:102B20000895882371F4772321F09850872B762F0E
:102B300007C0662311F499270DC09051862B70E0D1
:102B400060E02AF09A95660F771F881FDAF7880FE2
:102B50009695879597F908959F3F49F0915028F4ED
:102B6000869577956795B7959F5F80389F4F880FBB
:102B70009695879597F9089591505040660F771F65
:102B8000881FD2F708956CDEA0F0BEE7B91788F46D
:102B9000BB279F3860F41616B11D672F782F882742
:102BA000985FF7CF869577956795B11D9395963980
:082BB000C8F30895F894FFCF6B
:102BB80000000000000000000001020203030303FC
:102BC80004040404040404040505050505050505B5
:102BD8000505050505050505060606060606060695
:102BE800060606060606060606060606060606067D
:102BF8000606060606060606070707070707070765
:102C0800070707070707070707070707070707074C
:102C1800070707070707070707070707070707073C
:102C2800070707070707070707070707070707072C
:102C38000707070707070707080808080808080814
:102C480008080808080808080808080808080808FC
:102C580008080808080808080808080808080808EC
:102C680008080808080808080808080808080808DC
:102C780008080808080808080808080808080808CC
:102C880008080808080808080808080808080808BC
:102C980008080808080808080808080808080808AC
:102CA800080808080808080808080808080808089C
:082CB8000808080808080808D4
:00000001FF
